:100000001628FF3FFF3F8312031323088A002208AC
:100010008200080003208A110A128000840AA20AC2
:100020000319A30AF003031D0A280800831603130B
:100030009101073083129900C03083168500FF308C
:1000400087008312071A6D2885120516051485107E
:10005000A001A10103302102031D3028E830200255
:1000600003183628A00A0319A10A2A2885120516A2
:1000700005108514A001A10103302102031D4228AF
:10008000E830200203184828A00A0319A10A3C28D6
:100090008516051205108514A001A1010330210267
:1000A000031D5428E830200203185A28A00A031917
:1000B000A10A4E288516051205148510A001A1017C
:1000C00003302102031D6628E830200203186C2843
:1000D000A00A0319A10A60286D288719B828851677
:1000E000051205148510A001A10103302102031D92
:1000F0007B28E830200203188128A00A0319A10AEE
:1001000075288516051205108514A001A10103307C
:100110002102031D8D28E830200203189328A00A2D
:100120000319A10A87288512051605108514A00158
:10013000A10103302102031D9F28E830200203188B
:10014000A528A00A0319A10A9928851205160514E5
:100150008510A001A10103302102031DB128E83060
:1001600020020318B728A00A0319A10AAB28B8284F
:100170002128B928FF3FFF3FFF3FFF3FFF3FFF3FE1
:02400E00D400DC
:00000001FF
